:020000040000FA
:020000001428C2
:040002000034003492
:080008008B1807280E28F900EF
:100010000308FA00AF0F0E28AE0A8B107A0883008F
:10002000F90E790E8B1009008313831609308E00A8
:100030008F308100831287309F000330C000D030A2
:10004000C1008F30C200013090008E008F0085010A
:1000500086018316FF308500051085100511851176
:100060000130860083120C10831203130030AF009E
:10007000AE008F018E01BF018B100B168B170C1C6D
:1000800052280C10BF0A03303F02031C3F281221E4
:10009000D0300F02031C472812218F300E02031CA0
:1000A0004C28542812213F288B130F308500003034
:1000B0002F07031D64282E07031D6428A901AA0128
:1000C000AB01AC01842034282F08B3002E08B20005
:1000D0003C30B7000030B100B000B600B500B4004D
:1000E00064210430B7000030B100B000B600B500A4
:1000F000B40064212D30B7000030B600B500B40064
:100100007B210C22842034282908D0009920500813
:10011000D1002A08D00099205008D2002B08D00026
:1001200099205008D3002C08D00099205008D40002
:100130000800003050020319C22801305002031990
:10014000CA28023050020319D22803305002031982
:10015000DA28043050020319E2280530500203194E
:10016000EA28063050020319F2280730500203191A
:10017000FA280830500203190229093050020319E5
:100180000A290800D0175017D0165016D015501550
:10019000D0100800D0135017D0165012D0115011A3
:1001A000D0100800D0175017D0125016D01550118B
:1001B000D0140800D0175017D0165016D011501177
:1001C000D0140800D0135017D0165012D01150156B
:1001D000D0140800D0175013D0165016D011501557
:1001E000D0140800D0175013D0165016D015501543
:1001F000D0140800D0175017D0165012D01150113B
:10020000D0100800D0175017D0165016D015501522
:10021000D0140800D0175017D0165016D011501512
:10022000D0140800FF30850004302002031DA00A0E
:10023000AD010301290203192D142D1824292D10B5
:1002400001302002031946292D1827292D290301E1
:100250002A02031D2D292D1832292D1002302002CB
:1002600003194A292D1835293B2903012B02031DA7
:100270003B292D1840292D100330200203194E2947
:100280002D1004302002031952290800510886005D
:1002900005100800520886008510080053088600E3
:1002A00005110800540886008511A00108007E226F
:1002B0000318080030083406BC0047220310340835
:1002C0003006BC1F803E0800BC016822031C7B2254
:1002D00003180800562263221F30BD008E22380DFD
:1002E00003184722031C300D03180800BD0B6E29AC
:1002F0003C186B220800BC0137083604350434046E
:10030000003C031C6822031C7B2203180800BB016D
:10031000BA01B901B8018E221F30BD008E22340807
:100320003802031D9D2935083902031D9D29360811
:100330003A02031D9D2937083B02031CAF293708E9
:10034000BB023608031C360FBA023508031C350FF2
:10035000B9023408031C340FB80203103314BD0B68
:100360008E293C186B220800BC01682203109222DF
:1003700034083802031DC62935083902031D9D299A
:1003800036083A02031DC62937083B02031CD1294F
:10039000B30FD129B20FD129B10FD129B00A031956
:1003A00008003C186B220800300D03180800562284
:1003B0005F221030BD00BB0DBA0DB90DB80DB70DE1
:1003C000B60DB50DBB0DBA0DB90DB80DB70DB60D07
:1003D000B50D0314B30DB20DB10D31083502031D77
:1003E000F72932083602031DF72933083702031CA8
:1003F000042A3308B7023208031C320FB602310850
:10040000031C310FB502B3143310BD0BDB290310ED
:10041000B10CB20CB30C0800BC0168220318080030
:1004200097222030BD00B30DB20DB10DB00D2C30B0
:1004300084000A30BE00800D0A30000203188000DC
:100440008403BE0B1B2ABD0B132A3C185514031042
:100450000800BC002030BD00223084003C08BE00F3
:100460000A300310840A03188007800CBE0B322A5E
:10047000B00CB10CB20CB30CBD0B2C2A0008FF3E23
:10048000031C300D0318080055186B2208003708AC
:10049000B30736080318360FB20735080318350FAF
:1004A000B10734080318340FB00708003308BB0045
:1004B0003208BA003108B9003008B8000800B701A6
:1004C000B601B501B401B301B201B101B001080038
:1004D000300D031C080030088039B309B209B10996
:1004E000B009B30F782AB20F782AB10F782AB00A70
:1004F000BC0A30070800340D031C0800340880399A
:10050000B709B609B509B409B70F8B2AB60F8B2AFC
:10051000B50F8B2AB40ABC0A34070800B30DB20D1C
:10052000B10DB00DBB0DBA0DB90DB80D0800D50158
:10053000A301A401A501A601A701A801A901AA017F
:10054000AB01AC0108002130E000E00BA52A080057
:10055000C730E0000130E100B12A1F30E0004F3029
:10056000E100E00BB42AE10BB12AB62A0000080032
:02400E00103F61
:1042000046346F347234643475346C3461347434CD
:1042100073347A3461346D346D34653472346F3490
:1042200020344C34453444342D3465346C342E34CD
:1042300020344B3469347334653473347A347434D1
:0E424000653472346734613468346F347A3414
:1042600020342034763431342E3430342034203429
:104270004E3465346D3465347334683461347A3463
:1042800069342034473479346F3472346734793484
:00000001FF
